:1000000083160C308500003086008312E1288207B9
:100010003E344134413441343E34003410342034D1
:100020007F3400342734493449344934313422345C
:1000300041344934493436340C34143424347F3454
:1000400004347A3449344934493446343E344934EA
:1000500049344934263440344734483450346034C9
:1000600036344934493449343634323449344934E5
:1000700049343E3400348514000085102608A3005E
:10008000053098002308072086008620A30A980BD5
:10009000422808008514000085102708A3000530B9
:1000A00098002308072086008620A30A980B512871
:1000B00008008514000085102808A300053098006A
:1000C0002308072086008620A30A980B60280800D2
:1000D0008514000085102908A30005309800230826
:1000E000072086008620A30A980B6F280800851435
:1000F000000085102A08A300053098002308072077
:1001000086008620A30A980B7E2808009B0B862871
:1001100000308600051000000514080004309B0024
:100120009A0B90289B0B90280800910AA60AA60A11
:10013000A60AA60AA60A911C0800911D0800003014
:100140009100A600920AA70AA70AA70AA70AA70A67
:10015000921C0800921D080000309200A700930A2C
:10016000A80AA80AA80AA80AA80A931C0800931DAE
:10017000080000309300A800940AA90AA90AA90A55
:10018000A90AA90A941C0800941D080000309400D4
:10019000A900950AAA0AAA0AAA0AAA0AAA0A951CE2
:1001A0000800951D080000309500AA000800051DF4
:1001B000DA28DF289E1A08009E16952008009E1255
:1001C0000800003091009200930094009500A60072
:1001D000A700A800A900AA0060309C007720D720C3
:1001E0009C0BEE2820309C008E20D7209C0BF428FE
:1001F00060309C006820D7209C0BFA2820309C009F
:100200008E20D7209C0B002960309C005920D720DD
:100210009C0B062920309C008E20D7209C0B0C299B
:1002200060309C004A20D7209C0B122920309C0073
:100230008E20D7209C0B182960309C003B20D720B3
:100240009C0B1E29FF309C008E20D7209C0B24295C
:02025000EC2898
:00000001FF
